:030000000233EBDD
:0C33EB0078FFE4F6D8FD75816C023432E6
:100E29000A53746172743A20004950436F6E6E65BB
:100E390063745245510A004950436F6E6E6563747D
:100E4900003E432C562C52432CC0E4E0EFF2E5F06F
:100E590020D1E8EDEAEEEC49500A003E432C4D4121
:100E6900432C25303262583A25303262583A2530BF
:100E79003262583A25303262583A25303262583A4D
:100E890025303262582C4D414320E0E4F0E5F10A67
:100E9900003E432C5645522C20332E3120EEF220B1
:100EA90025732025732CC2E5F0F1E8FF2049502075
:100EB900ECEEE4F3EBFF0A004A616E203330203296
:100EC9003030380031313A31383A3030003E432C35
:100ED9004C442C50524F473A2020202020202020DB
:100EE90020202020202020202020202020202020F9
:100EF90020202020202020202020202020202020E9
:100F090020202020202020202020202020202020D8
:100F1900202020202020202020202020202CC4E058
:100F2900F2E020EFF0EEF8E8E2EAE828F4E0E9EB95
:100F3900290A003E2A2C312CCEF1EDEEE2EDFBE53B
:100F490020EFE0F0E0ECE5F2F0FB20F1E5F2E5E27C
:100F5900EEE3EE20E8EDF2E5F0F4E5E9F1E00A0070
:100F69003E412C4130312C2562752E2562752E2586
:100F790062752E2562752C495020E0E4F0E5F120D8
:100F8900E0E4E0EFF2E5F0E00A003E412C413032C6
:100F99002C2562752E2562752E2562752E256275A2
:100FA9002C495020E0E4F0E5F120EEF1ED2E20F19E
:100FB900E5F0E2E5F0E00A003E412C4130332C2512
:100FC90062752E2562752E2562752E2562752C494E
:100FD9005020E0E4F0E5F120F0E5E72E20F1E5F01E
:100FE900E2E5F0E00A003E412C4130342C256275DF
:100FF9002E2562752E2562752E2562752CCCE0F1A1
:10100900EAE020F1E5F2E80A003E412C4130352CB6
:101019002562752E2562752E2562752E2562752C21
:10102900D8EBFEE70A003E532C4130362C25627579
:101039002CC2F0E5ECFF20EEE6E8E42E20EAE2E837
:10104900F2E0EDF6E8E820282A3130ECF1290A002F
:101059003E2A2C312CC4EEEF2E20EFE0F0E0ECE537
:10106900F2F0FB20F1E5F2E5E2EEE3EE20E8EDF245
:10107900E5F0F4E5E9F1E00A003E422C5330312C69
:101089002562752CC6E4E0F2FC20E7E0EFF0EEF112
:10109900E020F1EEE5E4E8EDE5EDE8FF20EEF220F1
:1010A900F1E5F0E2E5F0E00A003E422C5330322C43
:1010B9002562752CCEE1ECE5ED20F120F1E5F0E2B9
:1010C900E5F0EEEC20E1E5E720EAE2E8F2E0EDF612
:1010D900E8E90A003E422C5330332C2562752CCFA7
:1010E900E5F0E5E7E0EFF3F1EA20EFF0E820EFEED5
:1010F900F2E5F0E520F1E2FFE7E820F120F1E5F083
:10110900E2E5F0EEEC0A003E422C5330342C256225
:10111900752CCDE5F220EFE5F0E5E4E0F7E820E411
:10112900E8E0E3EDEEF1F2E8EAE820E220F1E5F0AB
:10113900E2E5F00A003E422C5330352C2562752C2D
:10114900CAE0EDE0EB20F8E8F0EEEAEEE2E5F8E0DF
:10115900F2E5EBFCEDEEE3EE20EEE1ECE5EDE00A85
:10116900003E532C5330362C25303262582530320C
:101179006258253032625825303262582530326241
:101189005825303262582C4D414320E0E4F0E5F116
:1011990020F8E8F0EEEAEEE2E5F8E0F2E5EBFCED46
:1011A900EEE3EE20EEE1ECE5EDE00A003E454E44CB
:1011B9000A0044756D7058202020202030302030DE
:1011C9003120303220303320303420303520303651
:1011D900203037203038203039203041203042202B
:1011E90030432030442030452030460A003A003A46
:1011F90020000A0044756D704420202020203030E2
:101209002030312030322030332030342030352026
:1012190030362030372030382030392030412030E6
:10122900422030432030442030452030460A0045D2
:101239007272206B657900526420656570726F6DFA
:101249000A005264204D454D0A00526420436F64E0
:10125900650A0044656275674950204F4E0A00448B
:10126900656275674950204F46460A0044656275B4
:101279006755736572204F6E0A004465627567553C
:10128900736572204F46460A0044656275674D735F
:1012990067204F6E0A0044656275674D7367204F7A
:1012A90046460A00436F6E666967206C6F636B215F
:1012B9000A00577220656570726F6D0A00205361CC
:1012C900766520656570726F6D210A00457272201E
:1012D9004D414321004C6F61643E3E002A003C4170
:1012E90030313D003C4130323D003C4130333D001E
:1012F9003C4130343D003C4130353D003C413036C5
:101309003D003C21003C5330313D003C5330323DDF
:10131900003C5330333D003C5330343D003C5330A6
:09132900353D003C5330363D0017
:063C3E00016900016700AE
:10001E00C2AFC28E438910E4F58B758DB8D2ABD2C8
:04002E008ED2AF229D
:03001B000232BCF2
:1032BC00C0E0C083C082C0D0C2AFC28E758B007517
:1032CC008DB820060675A61E75A6E10567D202E527
:1032DC006960020569E568D3940140021568056CC4
:1032EC00E56C540F7050D20EE56C543F701AD2003E
:1032FC0090668DE0601204F0E0D394B4400A9080A4
:10330C00007480F0C2AF80FE906688E0600204F02A
:10331C00906104E0600214F090668EE0D39401405A
:10332C0003E014F0300502056AE56BD394644004A5
:10333C00D2068002056BE566D3940140021566D275
:0C334C008ED2AFD0D0D082D083D0E0323F
:1008B000C20B7D027C007F07123C218F25E5256459
:1008C0006060097D017F60123BB9D20BE4FDFC7FC3
:1008D0000B123C218F25E52530E6097D04E4FF124B
:1008E0003BDDD20B7D017C007F07123C218F25E58B
:1008F000257008FD7FFF123BB9D20B300B0312604D
:1009000000C2AFC288C2A8C2AA758900123358D2E9
:10091000AF90634C7403F0A374CCF0E490634BF09D
:10092000122E6F123C5AC2061238FA906358E0C376
:10093000940350037403F0D20BC20DC20CD2932067
:100940000B077E0E7F29122A7FE4906578F0120053
:100950001EC2AFA37408F09062B77424F0E4A3F051
:10096000906341E09062B9F0906342E09062BAF027
:10097000906343E09062BBF0906344E09062BCF00F
:10098000906345E09062BDF0906346E09062BEF0F7
:10099000756801E490657AF0C207C208C209C20A0C
:1009A000D2AF75A70775A61E75A6E1200B18AF2557
:1009B000FE7D03122C81E4FF1231727E637F78E4A6
:1009C000FB7D01122D7B90668DE060037401F0E4E5
:1009D000906104F0A37455F0A37481F0E4F56AE427
:1009E000F56B906104E070031218FF90668EE0B41E
:1009F00001119080007410F0E490668EF0D20BC26A
:100A00000CC20D908008E0F52530E405D207741083
:100A1000F0E52530E508D2099080087420F0E5253E
:100A200030E608D2089080087440F0E56AD3940359
:100A30004023908002E4F0908001F0908000F0E587
:100A40006AD39406400FE4F56AC20390657AF075A4
:100A500068011238FA9080A0E07003123679908015
:100A6000B8E070031236F39080D0E070031237DCE8
:100A7000908000E0701330071012297B906334EFF0
:100A8000F0D394004003120036908002E07006908C
:100A90008000E06005D2050209DFC205E4F56A9036
:100AA0006104E060030209DF30091212259B9063A4
:100AB00034EFF0D394004005E0FF123CFD20080322
:100AC000020C391222B8906334EFF070030209DF90
:100AD000906378E054BF247F7003020B9C14700372
:100AE000020B7424026003020BCF200B077E0E7FE3
:100AF00032122A7F300F74200371906350E0FF7030
:100B000006906354E06055906684E0FEB50722A32A
:100B1000E0FF906351E0B50718906686E0FF9063B0
:100B200052E0B5070C906687E0FF906353E06F607A
:100B30002B906354E06E7033906685E0FF906355B0
:100B4000E0B50727906686E0FF906356E0B5071B87
:100B5000906687E0FF906357E0B5070F90657A7461
:100B600001F0123D00756801020C3990668474FF33
:100B7000F0020C3990668DE060037401F090667CA1
:100B8000E0FF90637AE06F6003020C3990667CE0CE
:100B900004F0E4F568906578F0020C393003030244
:100BA0000C39906347E070030209DF1239ACD203BD
:100BB000E4F568906578F090668804F0E490667BD0
:100BC000F0A3F0200B737E0E7F40122A7F806A9084
:100BD000668DE060037401F0300352906378E0208A
:100BE000E74B90637AE0FF90667BE0FE6F600D90CC
:100BF0006683E07007EE146F703F801390667BE0B1
:100C000004F0906334E0FFD39404400312376D90F6
:100C100060007482F0A37401F090637AE090600247
:100C2000F07E607F007D0312357B0209DF300F0903
:100C300020030690668474FFF0200303020CEEE5A7
:100C400068706B12285AEF60207E647F7890647918
:100C5000E02404FD12357B906683E060030209DF27
:100C6000906358E0F5680209DF906688E0D3943C11
:100C7000403C906683E0703690668804F09062B6DF
:100C8000E0702B12300CE4906478F0A37412F090B2
:100C9000667CE090647AF0A374FDF090610763A233
:100CA0000190647C63A2017F12121E59809B123C4A
:100CB000EBEF60159060007483F0E4A3F07E607F3A
:100CC000007D0212357B0209DFE5686401600302E2
:100CD00009DF906578E004F0E0C394055003020C4E
:100CE00049C203E490657AF0123D000209DFE5682D
:100CF000640160030209DF90657AE014604624FE17
:100D00006042147003020DDC240460030209DFE476
:100D1000F56A200F1390657A7404F0906578E054BA
:100D200001F07568010209DF9080027410F0E49010
:100D3000657AF090657804F07568C890668474FFF1
:100D4000F00209DF906684E07003020DCB906478B6
:100D50007480F090647A7401F0E4A3F0A304F0A32B
:100D60007430F0A3747BF0E4F525747F2525F582BB
:100D7000E43464F583747DF074802525F582E434D1
:100D800064F583E4F0E5252407906479F07C667DC2
:100D90008490634CE0FAA3E0FB7F021234777E6418
:100DA0007F78E5252409FD12357B906683E0601B82
:100DB0001239ACD203E4F568906578F09066880447
:100DC000F0E490667BF0A3F00209DF90657A74048A
:100DD000F0906358E02432F5680209DF90800274D5
:100DE00010F0756803906578E06401FFF090657A13
:100DF0007401F0EF7019906354E06013FCA3E0FD00
:100E0000A3E0FEA3E0FF9066841217C10209DF9001
:100E10006350E0FCA3E0FDA3E0FEA3E0FF90668446
:080E20001217C10209DF80FE78
:010E280022A7
:10003600906379E0B444047F0180027F0090637886
:10004600E0B447047E0180027E00EE5F604A906362
:1000560041E090637AF0906342E090637BF09063B6
:1000660043E090637CF0906344E090637DF090639E
:1000760045E090637EF0906346E090637FF0906386
:10008600797452F09062B063A2019080A863A201D5
:100096007F06121E590208A6906334E0C3940850E6
:1000A600030208AF906341E0FF90637AE06F60035C
:1000B6000208AF906342E0FF90637BE06F6003024B
:1000C60008AF906343E0FF90637CE06F6003020833
:1000D600AF906344E0FF90637DE06F60030208AF7A
:1000E600906345E0FF90637EE06F60030208AF9087
:1000F6006346E0FF90637FE06F60030208AF9063A2
:1001060079E0B444159062B0E0B4FF0E63A20190AA
:1001160080A863A2017F06121E5990668DE06003D7
:100126007401F090668E7464F09063797452F09066
:100136006378E0646D60030202B37BFF7A0E794A4E
:100146001213947BFF7A0E7964906341E0F52EA337
:10015600E0F52FA3E0F530A3E0F531A3E0F532A3F7
:10016600E0F533121394752EFF752F0E7530C17599
:1001760031FF75320E7533CD7BFF7A0E799A1213E5
:10018600947BFF7A0E79D61213947BFF7A0F793C13
:100196001213947BFF7A0F7969906347E0F52EA3DB
:1001A600E0F52FA3E0F530A3E0F5311213947BFFC1
:1001B6007A0F7993906350E0F52EA3E0F52FA3E034
:1001C600F530A3E0F5311213947BFF7A0F79C190D5
:1001D6006354E0F52EA3E0F52FA3E0F530A3E0F598
:1001E600311213947BFF7A0F79EF90633DE0F52E81
:1001F600A3E0F52FA3E0F530A3E0F5311213947BCD
:10020600FF7A107912906339E0F52EA3E0F52FA35B
:10021600E0F530A3E0F5311213947BFF7A10792FC5
:10022600906358E0F52E1213947BFF7A10795912D9
:1002360013947BFF7A107982A20FE433F52E121302
:10024600947BFF7A1079B2906683E0F52E121394B0
:100256007BFF7A1079DD90668DE0F52E1213947B84
:10026600FF7A1179109062B6E0F52E1213947BFF97
:100276007A11793EA201E433F52E1213947BFF7AAC
:1002860011796A90667DE0F52EA3E0F52FA3E0F5DF
:1002960030A3E0F531A3E0F532A3E0F53312139471
:1002A600122B807BFF7A1179B51213942290637812
:1002B600E0644C70757E117FBB122A7F906380E0EC
:1002C600F526A3E0F527E4F5297E117FF6122A7FAD
:1002D6007D03AF27AE26122C817E117FF8122A7F6E
:1002E600E4F528852782852683E0FF74822528F594
:1002F60082E43463F583EFF00527E52770020526CF
:100306000528E528B410DC7E637F82E4FB7D1012AD
:100316002D7B7E117FFB122A7F0529E529C39410C8
:1003260040A77E117FFB122A7F22906378E0646CDF
:10033600705CF52A7E117FFD122A7FE4F529AF2A2B
:100346007E007D03122C817E117FF8122A7FE4F550
:1003560028A82AE6FF74822528F582E43463F5830B
:10036600EFF0052A0528E528B410E67E637F82E4CF
:10037600FB7D10122D7B7E117FFB122A7F0529E55E
:1003860029C3940840B87E117FFB122A7F2290630E
:1003960078E0644B7061F528746A2528F582E434A8
:1003A60063F583E06032746A2528F582E43463F5E8
:1003B60083E0F46023746A2528F582E43463F583C8
:1003C600E0FF74802528F582E43463F583E0B50701
:1003D600100528E528B408C09061047432F00208BC
:1003E600A69063787421F0300B030208A67E127F74
:1003F60038122A7F0208A6906378E0B4521A200BBE
:10040600077E127F40122A7F9063787472F07E63B3
:100416007F787D081234FB22906378E0644970454A
:10042600200B077E127F4B122A7F906380E0F52611
:10043600A3E0F527E4F528852782852683E0FF7467
:10044600822528F582E43463F583EFF00527E52756
:10045600700205260528E528B480DC7E637F787D5A
:100466008A1234FB22906378E064437079A3E064D7
:10047600527046200B077E127F53122A7F906380AC
:10048600E0F526A3E0F527E4F5288527828526836F
:10049600E493FF74822528F582E43463F583EFF054
:1004A6000527E527700205260528E528B480DB7EAA
:1004B600637F787D8A1234FB22906379E06457600B
:1004C600030208AF906380E0F526A3E0F527748267
:1004D6002528F582E43463AD82FC7B80AF27AE2607
:1004E600123AB50208A6906378E0644460030205F8
:1004F6007D906380E0FF644470030208A6EFB43188
:100506000CC20B7E127F5C122A7F0208A6906380C3
:10051600E0B4300CD20B7E127F68122A7F0208A646
:10052600906380E0B4320CD20C7E127F75122A7F63
:100536000208A6906380E0B4330CC20C7E127F835F
:10054600122A7F0208A6906380E0B4340CD20D7E96
:10055600127F92122A7F0208A6906380E0B4350CBF
:10056600C20D7E127F9F122A7F0208A6906380E04A
:10057600FF123C8D0208A6906104E07013200B0761
:100586007E127FAD122A7F9063787421F00208A64E
:100596009061047432F0906378E0FFB4510A908061
:1005A600007480F0C2AF80FEEF64577045200B07E1
:1005B6007E127FBB122A7F906381E0906334F0E461
:1005C600F528906334E0FFE528C39F40030208A6A0
:1005D60074822528F582E43463F583E0FF90638016
:1005E600E0252824AFF582E43461F583EFF0052891
:1005F60080D0906378E0645360030206AB200B075B
:100606007E127FC6122A7F906341E0FF9061B8E0B8
:100616006F703C906342E0FF9061B9E06F7030907C
:100626006343E0FF9061BAE0B50724906344E0FFBE
:100636009061BBE0B50718906345E0FF9061BCE0B0
:10064600B5070C906346E0FF9061BDE06F601690C1
:1006560063787421F0300B030208A67E127FD51250
:100666002A7F0208A6E4F528E4F56B74AF2528F581
:1006760082E43461F583E0FDAF28123B150528E5D9
:1006860028C394FE40E29080007480F0C2AFE490EC
:100696007FF0F0A3F0907FFD74AAF0A374FFF0A39F
:1006A6007455F080FE906378E0644F704C906380E0
:1006B600E0F526A3E0F527E5274526700A200B0777
:1006C6007E127FDE122A7F200B077E127FE5122A1A
:1006D6007FE4F52874822528F582E43463F583E007
:1006E600852782852683F00527E5277002052605DE
:1006F60028E528B480DE0208A6906378E0FFB445BA
:10070600279080007480F0906380E0FDA3E0907FE6
:10071600F0CDF0A3EDF0C2AF907FFD74AAF0A37404
:10072600FFF0A37455F080FEEF646560030208A62F
:10073600906380E0FFA3E0907FF0CFF0A3EFF0E4BA
:10074600F526F527D3907FF1E09527907FF0E09589
:10075600264021E4F56B2527FFE5263478FE7B80CD
:10076600AD27AC26123AB574802527F527E4352641
:10077600F52680D07E127FE71235FBEF4E60201201
:100786000003906347EFF0120003906348EFF01206
:100796000003906349EFF012000390634AEFF07E86
:1007A600127FED1235FBEF4E60201200039063506E
:1007B600EFF0120003906351EFF0120003906352C2
:1007C600EFF0120003906353EFF07E127FF31235C1
:1007D600FBEF4E6020120003906354EFF01200030B
:1007E600906355EFF0120003906356EFF01200038A
:1007F600906357EFF07E127FF91235FBEF4E6020C3
:1008060012000390633DEFF012000390633EEFF099
:1008160012000390633FEFF0120003906340EFF085
:100826007E127FFF1235FBEF4E60201200039063AD
:1008360039EFF012000390633AEFF0120003906371
:100846003BEFF012000390633CEFF07E137F05123E
:1008560035FBEF4E600812389D906358EFF0E4F5D3
:1008660028E4F56BE52804FF74392528F582E4347D
:1008760063F583E0FD123B150528E528C394434044
:10088600E09080007480F0C2AFE4907FF0F0A3F0B7
:10089600907FFD74AAF0A374FFF0A37455F080FE58
:0908A6007E637F787D081234FBAB
:0108AF002226
:103A7D00AE07EEC39430400BEED394395005EE24CF
:103A8D00D0FF22EEC39461400BEED394665005EE49
:103A9D0024A9FF22EEC39441400BEED3944650056A
:083AAD00EE24C9FF22AF06223E
:103C76009062AFE004F070069062AEE004F09062ED
:073C8600AFE0FF123B3F22FB
:10000300123C76123A7DEFC454F0FEC006123C76E1
:08001300123A7DD0E02FFF221C
:10389D00E4906A3EF0123C76906A3FEFF0C39430AC
:1038AD004018E0FFD394395011906A3EE02407F59B
:1038BD0082E43461F583EFF08011906A3EE02407D5
:1038CD00F582E43461F583E4F0800C906A3EE00407
:1038DD00F0E0D3940840BE753100753200753300A9
:0C38ED00E4F5347B017A617907122114A4
:0138F90022AC
:0435FB008E2B8F2C58
:1035FF009062AEE4F0A374FFF0123C76EF6067F4D4
:10360F006064852C82852B83E493B507EC752D01BF
:10361F00E52C252DF582E4352BF583E493601E9080
:10362F0062AFE0252DFF123B3FE52C252DF582E4FF
:10363F00352BF583E493B50704052D80D3E52C25B1
:10364F002DF582E4352BF583E49370ADE52D24FF42
:10365F00FFE434FFFE9062AFE02FF09062AEE03EE9
:09366F00F07E007F0122E4FEFF61
:01367800222F
:102E6F007E137F0B1235FBEF4E70037F01227E1313
:102E7F007F0E1235FBEF4E600C123C76EF24D02400
:102E8F00FF920F8002D20F7E137F141235FBEF4E8D
:102E9F00600C123C76EF24D0906683F08005E490AE
:102EAF006683F07E137F1A1235FBEF4E600C123CD7
:102EBF0076EF24D090668DF08005E490668DF07EDD
:102ECF00137F201235FBEF4E600C123C76EF24D0AF
:102EDF009062B6F08005E49062B6F07E137F261202
:102EEF0035FBEF4E600C123C76EF24D024FF92019D
:102EFF008002C20190634163A20190667D63A201CB
:102F0F007F06121E5930013B7E137F2C1235FBEFCB
:102F1F004E603012000390667DEFF0120003906652
:102F2F007EEFF012000390667FEFF01200039066C1
:102F3F0080EFF0120003906681EFF01200039066AD
:062F4F0082EFF07F00227A
:1039FD00906579E0C3947C503D906579E0FE04F0CC
:103A0D0074B72EF582E43462F583EFF0BF0A279088
:103A1D006579E0FF04F074B72FF582E43462F58325
:103A2D00E4F0906579E0FF12321C9065797408F02E
:073A3D009062B8E004F022E2
:1038FA009080007480F090633963A201F583F582A9
:10390A0063A2017F08121E5990634163A20190804D
:10391A008863A2017F0A121E59908092E4F0A37470
:10392A0032F0A37401F090634BE0FF9080B1F09005
:10393A0080E1EFF09080957455F0A3F090800074C8
:09394A0001F090800974F0F022F4
:10367900908009E04410F09080A0E0706C9080A1E7
:103689007482F09080A874FFF0A3F0A3F0A3F07FF8
:10369900039080AEEFF07FCBA3EFF07F039080AC77
:1036A900EFF0A374CBF09080007402F0906A2E12B0
:1036B90017CD00000000906A2EE0908040F0906ADB
:1036C9002FE0908041F0906A30E0908042F0906A5B
:1036D90031E0908043F0A3E4F0A3F0A3F0A3F090CD
:0936E9008018F0A3F0A3F0A3F097
:0136F20022B5
:1037DC00908009E04440F09080D17482F090634C6A
:1037EC00E0FF9080DEF090634DE0FF9080DFF09082
:1037FC0080027402F0906A321217CD000000009023
:10380C006A32E0908058F0906A33E0908059F090E2
:10381C006A34E090805AF0906A35E090805BF0A3B7
:10382C00E4F0A3F0A3F0A3F0908030F0A3F0A3F0A9
:02383C00A3F0F7
:01383E002267
:1036F300908009E04420F09080B8E0706C9080B92D
:103703007482F07F039080C6EFF07FCDA3EFF07F4C
:10371300039080C4EFF0A374CDF09080C074FFF0E9
:10372300A3F0A3F0A3F09080017402F0906A361224
:1037330017CD00000000906A36E090804CF0906A4C
:1037430037E090804DF0906A38E090804EF0906AB8
:1037530039E090804FF0A3E4F0A3F0A3F0A3F0903E
:093763008024F0A3F0A3F0A3F010
:01376C00223A
:103477008C268D27A907EAFDE975F018A424ACFF6F
:10348700E5F034808F82F583EDF0EBFDE975F018F8
:10349700A4FFAEF024ACFBEE34808B82F583A3ED62
:1034A700F08527828C83E0FDEF24A8FFEE3480FEB1
:1034B7008F82F583EDF08527828C83A3E08F828E40
:1034C70083A3F0852782852683A3A3E0FDE975F012
:1034D70018A424A8FFE5F03480FE8F82F583A3A308
:1034E700EDF08527828C83A3A3A3E08F828E83A32D
:0434F700A3A3F02279
:0634FB008D2BAB07AA06B1
:10350100908000E020E572906A2EE0FCA3E0FDA32C
:10351100E0FEA3E0F52F8E2E8D2D8C2CAE02AF0395
:103521008E838F8263A201E52E540744C0F5838503
:103531002F8263A201AF2B121ECBE4FCFDFEE52F0F
:10354100252BF52FEE352EF52EED352DF52DEC3500
:103551002CF52C908040E52CF0A3E52DF0A3E52E71
:10356100F0A3E52FF09080007420F0AF2FAE2EADC8
:093571002DAC2C906A2E1217C13A
:01357A00222E
:06357B008D26AB07AA0635
:10358100908002E020E572906A32E0FCA3E0FDA3A6
:10359100E0FEA3E0F52A8E298D288C27AE02AF0329
:1035A1008E838F8263A201E529540744D0F5838578
:1035B1002A8263A201AF26121ECBE4FCFDFEE52A9E
:1035C1002526F52AEE3529F529ED3528F528EC359E
:1035D10027F527908058E527F0A3E528F0A3E529F2
:1035E100F0A3E52AF09080027420F0AF2AAE29AD55
:0935F10028AC27906A321217C1C0
:0135FA0022AE
:023172008F26A6
:10317400908001E030E5037F0022906A36E0FCA3F2
:10318400E0FDA3E0FEA3E0F52A8E298D288C27908C
:10319400667D63A201E529540744C8F583852A8224
:1031A40063A2017F06121EE1E52A2406F52AE4350E
:1031B40029F529E43528F528E43527F52790657B9A
:1031C40063A201E529540744C8F583852A8263A2D2
:1031D40001AF26121EE1E4FCFDFEE52A2526F52AB0
:1031E400EE3529F529ED3528F528EC3527F5279016
:1031F400804CE527F0A3E528F0A3E529F0A3E52A10
:10320400F09080017420F0AF2AAE29AD28AC27904D
:073214006A361217C1AF2654
:01321B002290
:10297B009081E0E0F5260526052605260526052689
:10298B0005260526052605260526908010E0F52947
:10299B00A3E0F52AA3E0F52BA3E0F52C9081E1E071
:1029AB00F5260526052605260526052605260526D4
:1029BB00052605260526908014E0F52DA3E0F52EBF
:1029CB00A3E0F52FA3E0F530E52FB52B08E530B5E7
:1029DB002C037F0022E4F526E52F540744E0F58312
:1029EB0085308263A20190637863A2017F08121F76
:1029FB001190637A63A2019062B063A2017F061209
:102A0B001E59906378E0F527A3E0F528E4F52690AE
:102A1B006378E0702AA3E024F8F526E52F540744E9
:102A2B00E0F58385308274082582F582E43583F5E1
:102A3B008363A20190637863A201AF26121F11AECC
:102A4B0027E4FCFDE5302528F530E52F3EF52FED8D
:102A5B00352EF52EEC352DF52D908014E52DF0A3AC
:102A6B00E52EF0A3E52FF0A3E530F0908000744045
:032A7B00F0AF2693
:012A7E002235
:1022B8009081E6E0F526052605260526052605264D
:1022C80005260526052605260526908028E0F529F9
:1022D800A3E0F52AA3E0F52BA3E0F52C9081E7E035
:1022E800F52605260526052605260526052605269E
:1022F80005260526052690802CE0F52DA3E0F52E71
:10230800A3E0F52FA3E0F530E4F526E52FB52B0A79
:10231800E530B52C05C208022412E52F540744F015
:10232800F58385308263A20190637863A2017F08F8
:10233800121F11906378E0F527A3E0F528E52845FA
:102348002770099080027410F07F0022906684E064
:10235800FFF4602D90637AE06F7076906685E0FFF9
:1023680090637BE06F706A906686E0FF90637CE024
:102378006F705E906687E0FF90637DE06F602280FB
:102388005090637AE0906684F090637BE090668575
:10239800F090637CE0906686F090637DE0906687BD
:1023A800F0906378E0702AA3E024F8F526E52F542E
:1023B8000744F0F58385308274082582F582E43578
:1023C80083F58363A20190637863A201AF26121F8D
:1023D80011AE27E4FCFDE5302528F530E52F3EF564
:1023E8002FED352EF52EEC352DF52DAF2CAE2BAD72
:1023F8002AAC29AB30AA2FA92EA82DD31217B0408A
:10240800099080027410F07F002290802CE52DF056
:10241800A3E52EF0A3E52FF0A3E530F09080027439
:0424280040F0AF26AB
:01242C00228D
:10259B009081E3E0F526052605260526052605266A
:1025AB000526052605260526052690801CE0F5291F
:1025BB00A3E0F52AA3E0F52BA3E0F52C9081E4E052
:1025CB00F5260526052605260526052605260526B8
:1025DB00052605260526908020E0F52DA3E0F52E97
:1025EB00A3E0F52FA3E0F530E4F526E52FB52B0A94
:1025FB00E530B52C05C2090226E6E52F540744E861
:10260B00F58385308263A20190600463A2017F0E83
:10261B00121F27906004E0F527A3E0F52890600CCB
:10262B00E0FFF4604590667DE0FEEF6E706EA3E018
:10263B00FF90600DE06F706490667FE0FF90600E1E
:10264B00E06F7058906680E0FF90600FE06F704C09
:10265B00906681E0FF906010E06F7040906682E0C2
:10266B00FF906011E06F60048032D2D9906004E07B
:10267B00702AA3E024F2F526E52F540744E8F583EE
:10268B00853082740E2582F582E43583F58363A24F
:10269B000190600463A201AF26121F27AE27E4FC52
:1026AB00FDE5302528F530E52F3EF52FED352EF5E0
:1026BB002EEC352DF52DAF2CAE2BAD2AAC29AB3036
:1026CB00AA2FA92EA82DD31217B05006E5284527FF
:1026DB0070099080017410F07F0022908020E52D0E
:1026EB00F0A3E52EF0A3E52FF0A3E530F0908001E9
:0526FB007440F0AF2661
:0127000022B6
:042A7F008E2B8F2CDF
:102A8300E4F52DF52E908000E030E511052EE52EBE
:102A93007002052DD394E8E52D940340E89080005F
:102AA300E030E503022B7F906A2EE0FCA3E0FDA358
:102AB300E0FEA3E0F5328E318D308C2FE532FFE559
:102AC300315407FEE42FF52EEE34C0F52D852E820A
:102AD300F5837423F0052EE52E7002052D532DC7C3
:102AE300F582852D83740AF0052EE52E7002052DDF
:102AF300532DC790634163A201852D83852E826385
:102B0300A2017F06121ECB7406252EF52EE4352D69
:102B1300F52D852B83852C8263A201852D83852E3C
:102B23008263A201121EAFE4FCFDFE906A2EE0F860
:102B3300A3E0F9A3E0FAA3E02FFFEE3AFEED39FD9F
:102B4300EC38FCEF2408FFE43EFEE43DFDE43CFCEE
:102B5300906A2E1217C1906A2EE0908040F0906A1E
:102B63002FE0908041F0906A30E0908042F0906ACC
:0C2B730031E0908043F09080007420F06E
:012B7F002233
:062D7B008E2B8F2C8D2D24
:102D8100E4F52EF52F908000E030E511052FE52FB9
:102D91007002052ED394E8E52E940340E89080005C
:102DA100E030E503022E6E906A2EE0FCA3E0FDA365
:102DB100E0FEA3E0F5338E328D318C30E533FFE553
:102DC100325407FEE42FF52FEE34C0F52E852F8205
:102DD100F5837423F0052FE52F7002052E532EC7BE
:102DE100F582852E83EBF0052FE52F7002052E531A
:102DF1002EC790634163A201852E83852F8263A232
:102E0100017F06121ECB7406252FF52FE4352EF512
:102E11002E852B83852C8263A201852E83852F82AB
:102E210063A201AF2D121ECB7408252DF52DFFE4F1
:102E3100FCFDFEE5332FF533EE3532F532ED35315C
:102E4100F531EC3530F530908040E530F0A3E531D7
:102E5100F0A3E532F0A3E533F09080007420F0AFE9
:0D2E610033AE32AD31AC30906A2E1217C185
:012E6E002241
:02321C008F3FE2
:10321E00E4F540F541908000E030E5110541E541CF
:10322E0070020540D394E8E540940340E890800096
:10323E00E020E579906A2EE0FCA3E0FDA3E0FEA37A
:10324E00E0F5458E448D438C42E545FFE544540739
:10325E00FEE42FF541EE34C0F5409062B763A20153
:10326E0085408385418263A201AF3F121ECBE4FCF1
:10327E00FDFEE545253FF545EE3544F544ED354378
:10328E00F543EC3542F542908040E542F0A3E5432C
:10329E00F0A3E544F0A3E545F09080007420F0AF74
:0D32AE0045AE44AD43AC42906A2E1217C1EC
:0132BB0022F0
:062C81008E2E8F2FAB0523
:102C8700E4F530F531908000E030E5110531E531AC
:102C970070020530D394E8E530940340E890800053
:102CA700E030E503022D7A906A2EE0FCA3E0FDA355
:102CB700E0FEA3E0F5358E348D338C32E535FFE544
:102CC700345407FEE42FF531EE34C0F530853182F8
:102CD700F5837423F00531E531700205305330C7B1
:102CE700F582853083EBF00531E5317002053090D0
:102CF700634163A20185308385318263A2017F0628
:102D0700121ECB74062531F531E43530F5305330DA
:102D1700C7E52E853182853083F00531E5317002B4
:102D270005305330C7F582853083E52FF00531E54F
:102D370031700205305330C7E535240AF535E435DF
:102D470034F534E43533F533E43532F532908040E9
:102D5700E532F0A3E533F0A3E534F0A3E535F090D1
:102D670080007420F0AF35AE34AD33AC32906A2EAC
:032D77001217C16F
:012D7A002236
:10335800E4F526E52604FF123B3F74392526F5825D
:10336800E43463F583EFF00526E526C3943F40E394
:10337800E4F526E526247FFF123B3F742F2526F52A
:1033880082E43461F583EFF0742F2526F582E43466
:1033980061F583E0FF6003B4FF1D742F2526F582D5
:1033A800E43461F5837420F074302526F582E43422
:1033B80061F583E4F080090526E526C3948040B3CF
:1033C800E49061AEF0F526AF26123B3F74AF252698
:1033D800F582E43461F583EFF00526E526C394FE13
:0233E80040E5BE
:0133EA0022C0
:103C0100E4FDFCC3ED9FEC9E5015E4FBFA0BBB00F9
:0F3C1100010ABA01F8BB90F50DBD00010C80E46B
:013C20002281
:0D3CC4004390014390025390FE5390FD2267
:0D3CD1005390FD5390FE439002439001225A
:0E3CB5005390FD439002E5905408FF5390FD9C
:013CC30022DE
:0D3CDE005390FD4390014390025390FD224E
:073CF600AE071FEE70FA2279
:023AE900AD0727
:103AEB00E4FC5390FDEDA804088002C333D8FC30EE
:103AFB00E70543900180035390FE7F05123CF6438C
:093B0B0090020CBC08DC5390FD93
:013B1400228E
:103B6900E4FF5390FD7E07439002E59030E00D7429
:103B790001A806088002C333D8FC42075390FD1EF2
:083B8900C3EE6480948050DF5C
:013B91002211
:103B1500AB05AA07123CC47FA0123AE9123CB5AF27
:103B250002123AE9123CB5AF03123AE9123CB5125A
:0A3B35003CD17F0A7E00123C012201
:023B3F00AB07D2
:103B4100123CC47FA0123AE9123CB5AF03123AE924
:103B5100123CB5123CC47FA1123AE9123CB5123BAA
:073B610069123CDE123CD1A9
:013B6800223A
:023AB5008B2B59
:103AB700A2AF921EC2AF85A22C53A2FE8E838F8225
:103AC70005A28C838D827409121F55E52B53A2FE24
:103AD70043A220121F5753A2DF852CA2A21E92AF2A
:013AE700FFDF
:013AE80022BB
:103C2100A2AF921EC2AF8C838D82EF121F5543A2A9
:0C3C310020121F5753A2DFA21E92AFFF0B
:013C3D002264
:023BB9008F2655
:103BBB00A2AF921EC2AFE4F5838D827406121F551D
:103BCB00E52643A220121F5753A2DFA21E92AF7FFE
:013BDB0001E8
:013BDC0022C6
:023BDD008F2631
:103BDF00A2AF921EC2AFE4F5838D82740A121F55F5
:103BEF00E52643A220121F5753A2DFA21E92AF7FDA
:013BFF0001C4
:013C000022A1
:101D7E00A907E7FFA805EF93C3966008403B74FCE4
:101D8E002FFF80F00F08EF93C3966008402B74FB73
:101D9E002FFF80E00F08EF93C3966008401B74FA84
:101DAE002FFF80D00F08EF93D3966008400B74F985
:101DBE002FFF80C01F1F1F1F1FEF54FEF80303F7D6
:101DCE00E893FC08E893FD08E893FE08E893FF22E9
:101DDE0009E993C39D6008402974FB29F980F10934
:101DEE00E993C39E6008401A74FA29F980E209E962
:101DFE0093D39F6008400B74F929F980D3191919F0
:101E0E001919E9C313C313FF22740093F8ECC39896
:101E1E004024701F740193F8EDC398401970147428
:0E1E2E000293F8EEC398400E7009740393F807
:101E3C00EFC39840037F00227F0122EDF8E6F00803
:101E4C00A3DFFA22EDF8E0F608A3DFFA22E0A363A1
:101E5C00A201F0A363A201DFF475A2002263A20128
:101E6C00F0A363A20122E0A363A201F0A363A20189
:101E7C00E0A363A201F0A363A201E463A201F0A3B7
:101E8C0063A201DFE175A20022E0A363A2016DFE53
:101E9C00936CFDEE058393FC158363A201DFEA7559
:101EAC00A200227F00E493A363A201F00F600CA3B5
:101EBC00E583C2E3F58363A20180EA75A20022E008
:101ECC00A363A201F0A3E583C2E3F58363A201DF60
:101EDC00EE75A20022E0A363A201F0A3E583C2E4A5
:101EEC00D2E3F58363A201DFEC75A20022E0A363C9
:101EFC00A201F0A3E58344F8C2E5F58363A201DFF8
:101F0C00EC75A20022E583C2E3F583E0A363A20192
:101F1C00F0A363A201DFEE75A20022E583C2E4D236
:0A1F2C00E3F583E0A363A201F0A334
:101F360063A201DFEC75A20022E58344F8F583E095
:101F4600A363A201F0A363A201DFEE75A20022F94A
:101F560022C002C004C00612FFF0D006D004D00290
:011F66002258
:103C8D00BF360BD217E4F547F548F563F564BF373A
:043C9D0002C2172226
:10383F00C2A9438902906A29E0FFF58C8F8A75D956
:10384F000475DA4875DB3175DC4975DD4975DE3194
:10385F00E4F5E9F5F9F5EBF5FB906A27E0601675ED
:10386F00EC1075ED10E4F5FCF5FD755F08755D1056
:10387F00755E01801375EC8075ED80E4F5FCF5FD48
:0E388F00755F80F55D755E10E4F5EEF5FE22C6
:103A4400E4FEAF8CEFFD906A28E07003A3E06D60A4
:103A54000512383F7E01E5D920E2057E0212383F87
:103A6400E58920E10512383F7E03D28C75D8407574
:083A7400B740D2AED2AFAF069D
:013A7C002227
:0300330002242D77
:0B242D00C0E0C083C082C0D075D008A2
:10243800C2AF30DC56C3E5EC95EEC3955F5012E5AC
:102448005E25ECF5EC30D70405FC801685FCFC8095
:1024580011C3E5EC955EF5EC30D70415FC800385D7
:10246800FCFC301724854882854783E590F00548B1
:10247800E54870020547F582854783E5EEF0054893
:10248800E5487002054753470FC2DC30D929301799
:1024980024854882854783E590F00548E548700221
:1024A8000547F582854783E5EBF00548E548700266
:1024B800054753470FC2D930DA5AE55D700405FC69
:1024C8008010E55D25ECF5EC30D70405FC8003852C
:1024D800FCFCE5495480F546E54925E0F549309787
:1024E80002054920160363490130270FE549B56500
:1024F80021755B00756000C22780170560E5605490
:1025080007700F53603FE560131313541F244BF8F3
:10251800A649C2DA30DB71E55D700405FD8010E57F
:102528005D25EDF5ED30D70405FD800385FDFDE55E
:1025380061655C6029E55C54077013E55C1313134F
:10254800541F2453F8E6F54A201403634AFFE54A6A
:10255800339296E54A25E0F54A055C535C3FB29212
:10256800301723854882854783E590F00548E5487C
:1025780070020547F582854783E4F00548E5487011
:0A25880002054753470FC2DBD2AF34
:09259200D0D0D082D083D0E03219
:101B56004241554400575F4D4F44454D00494E564E
:101B66005F52454300494E565F5452414E53004919
:101B76004E565F414C4C004D4150424F415244003D
:101B8600554E49544D00003E2A2C312CCFE0F0E052
:101B9600ECE5F2F0FB20F1E8EDF5F0EEEDEDEEE32D
:101BA600EE20EFEEF0F2E00A003E4C2C4230312CF3
:101BB600256C752CD1EAEEF0EEF1F2FC20EEE1ECAC
:101BC600E5EDE02C35302C3130302C3230302C33F2
:101BD60030302C3630302C313230302C32343030FC
:101BE6002C343830300A003E422C4731302C2562E6
:101BF600752CC8EDE2E5F0F1E8FF20EDE020EFF00E
:101C0600E8B8ECE50A003E422C4731312C256275D6
:101C16002CC8EDE2E5F0F1E8FF20EDE020EFE5F07D
:101C2600E5E4E0F7E50A003E422C4730322C256217
:101C3600752CD3EFF0E0E2EBE5EDE8E520EFEEF210
:101C4600EEEAEEEC2020285254532D435453290A31
:101C5600003E532C4730332C256C752CC7E0E4E549
:101C6600F0E6EAE020F1F2E0F0F2E020EFE5F0E560
:101C7600E4E0F7E828ECF1290A003E532C4730331C
:101C86002C256C752C202AE7E0E4E5F0E6EAE02056
:101C9600F1F2E0F0F2E020EFE5F0E5E4E0F7E82825
:101CA600ECF1290A003E2A2C312CC0E4E0EFF2E5E3
:101CB600F020F1E8EDF5F0EEEDEDEEE3EE20EAE0F2
:101CC600EDE0EBE02E20CFF0EEF2EEEAEEEB20D2E6
:101CD600CC3531320A003E422C5430312C25627507
:101CE6002CC2FBE2EEE420D2D120EDE020F9E8F2AE
:101CF6000A003E422C5430322C2562752CD0E5E683
:101D0600E8EC20554E49544D0A003C21003C423037
:101D1600313D003C4731303D003C4731313D003CD0
:101D26004730323D003C4730333D003C5430313D76
:101D3600003C5430323D000AC3EEF2EEE220EFE002
:101D4600EAE5F220EA20EEF2EFF0E0E2EAE50A0048
:101D5600FF1B56FF1B5BFF1B63FF1B6BFF1B75FF08
:101D66001B7DFF1B86FF1B8C0008040C020A060E57
:081D76000109050D030B070F25
:103C440052668F0000000000000000000000000029
:053C540000000000006B
:103CA100EF540F901D6E93FEC454F0FEEFC4540FF9
:043CB100932EFF222D
:033CFD008F2622ED
:023953008F2EB5
:10395500906926E0FF04F074A22FF582E43466F541
:10396500837420F0E4FFEFC39D503BE52E75F00313
:10397500A42456F582E4341DF583E493FB74019386
:10398500FA740293F98F827583001216A7FE906967
:1039950026E024A2F582E43466F583EEF00F906903
:0639A50026E004F080C0E2
:0139AB0022F9
:103B9200742F2FF582E43461F583E0FE6420601611
:103BA200906926E0FD04F074A22DF582E43466F5F6
:063BB20083EEF00F80DA43
:013BB80022EA
:101F6700200B09AF267E007D03122C81E4906926A1
:101F7700F0F526E52675F003A42456F582E4341D12
:101F8700F583E493FB740193FA740293F912168EA6
:101F97007003022113E4F528F529F527742F252767
:101FA700F582E43461F583E0FF700302210EE52634
:101FB70075F003A42456F582E4341DF583E493FBFE
:101FC700740193FA740293F98528827583001216B7
:101FD700A7FEEFB506087529010528022109E5299D
:101FE7007003022109EE6003022104AD28AF261217
:101FF7003953E526B40700400302210E90200AF862
:1020070028287302201F0220B90220EE0220F202C4
:1020170020F60220FC022100AF27123B92742F25E5
:1020270027F9E43461FA7B01C0031B8B3175320059
:10203700753300E4F534D0031221148F2D8E2C8DC7
:102047002B8C2AE4FFFEFDFCAB2DAA2CA92BA82A7A
:10205700C31217B06022AB2DAA2CA92BA82AE47FA4
:10206700207E1CFDFC1217101217A2906A28EEF0B2
:10207700A3EFF0E4906A27F0E47FB07E04FDFCABA9
:102087002DAA2CA92BA82AD31217B0407A906A2719
:102097007401F0AB2DAA2CA92BA82A7F007EC2FDC4
:1020A7007C001217101217A2906A28EEF0A3EFF027
:1020B7008055AF27123B92D21A742F2527F9E434A3
:1020C70061FA7B01C0031B8B31753200753300E465
:1020D700F534D0031221148F2D8E2C8D2B8C2A9042
:1020E70066A1E52DF08020D216801CD2148018D26C
:1020F70016D2148012D215800ED210800AE4F52968
:0C210700F5280527021FA30526021F7AF9
:0121130022A9
:102B80007BFF7A1B798D121394906A27E0602FA344
:102B9000E0FEA3E0FFC3E49FFFE49EFEAB07FAE480
:102BA000F9F8FF7EC27D01FC1217108F318E308D37
:102BB0002F8C2E7BFF7A1B79AF121394802F906A93
:102BC00028E0FEA3E0FFC3E49FFFE49EFEAB07FA0C
:102BD000E4F9F87F207E1CFDFC1217108F318E3037
:102BE0008D2F8C2E7BFF7A1B79AF1213947BFF7A8B
:102BF0001B79EDA216E433F52E1213947BFF7A1C99
:102C0000790CA214E433F52E1213947BFF7A1C790D
:102C10002DA21AE433F52E121394301A1F7BFF7A7B
:102C20001C79579066A1E075F00AA4FFAEF0E48F1E
:102C3000318E30F52FF52E121394801D7BFF7A1CF8
:102C400079809066A1E075F00AA4FFAEF0E48F31C0
:102C50008E30F52FF52E1213947BFF7A1C79AB1270
:102C600013947BFF7A1C79DCA215E433F52E121342
:102C7000947BFF7A1C79F8A210E433F52E1213949A
:012C80002231
:102701007E1D7F101235FBEF4E70037F01227E1D6F
:102711007F131235FBEF4E70030227A812389D90EC
:102721006A3A1217C1E4FFFEFDFC906A3AE0F8A391
:10273100E0F9A3E0FAA3E0FBC31217B06025906AA9
:102741003AE0F8A3E0A3E0A3E0E47F207E1CFDFCD7
:102751001217101217A2906A28EEF0A3EFF0E4907E
:102761006A27F0E47FB07E04FDFC906A3AE0F8A3AA
:10277100E0F9A3E0FAA3E0FBD31217B04038906A66
:10278100277401F0906A3AE0F8A3E0A3E0A3E07FA8
:10279100007EC27D017C001217101217A2906A28D8
:1027A100EEF0A3EFF0800F906A2874FFF0A374B8E5
:1027B100F0E4906A27F07E1D7F191235FBEF4E6021
:1027C1000C123C76EF24D024FF92168002C2167EB2
:1027D1001D7F1F1235FBEF4E600C123C76EF24D0AB
:1027E10024FF92148002C2147E1D7F251235FBEF57
:1027F1004E600C123C76EF24D024FF921A8002C264
:102801001A7E1D7F2B1235FBEF4E601312389DE4AB
:102811007B0AFAF9F81217109066A1EFF08005E42F
:102821009066A1F07E1D7F311235FBEF4E600C12D8
:102831003C76EF24D024FF92158002C2157E1D7FC5
:10284100371235FBEF4E600C123C76EF24D024FF9B
:0828510092108002C2107F000A
:01285900225C
:103C5A00906A2874FFF0A374B8F0E4906A27F0120F
:0C3C6A002701EF6003121F6712383F2291
:1039AC0075657FC213D218C21DD227C21BC211C2A9
:1039BC001CE49067E2F0906925F0FFEF25E024E32A
:1039CC00F582E43468AD82F5168D17F583E4F00FBB
:1039DC00BF20E8E4FFEF25E02427F582E43469AD4D
:1039EC0082F5168D17F583E4F00FBF80E8123A4488
:0139FC0022A8
:10376D0020106990637CE0FE30E713541F25E024A0
:10377D00E1F582E43468AD82F5168D1780189063FB
:10378D007CE0540F75F010A42417F582E5F0346930
:10379D00AD82F5168D17E4FEEF24FBFDEEC39D50B3
:1037AD002B851782851683E04480F0747D2EF5827B
:1037BD00E43463F583E0851782851683A3F07402E4
:0E37CD002517F517E43516F5160E80CCD21C24
:0137DB0022CB
:1030C100906925E004F024DF700302316BE0FF25F5
:1030D100E024E1F582E43468AD82F5168D17F583BD
:1030E100E060DD0513E513AC127002051214F582E0
:1030F1008C83747FF0EF2480FF0513E513AC12700D
:1031010002051214F5828C83EFF0851382851283F8
:10311100F030D003E0F4F00513E5137002051285D9
:103121001782851683A3E0FF0513E513AC12700225
:10313100051214F5828C83EFF0851782851683A31F
:10314100E06455851382851283F020D012851782A1
:10315100851683A3E0F46455851382851283F005F7
:1031610013E513700205127F0522E4906925F0FF33
:01317100223B
:102F55009067E2E004F024EF7003023005E0FF75AE
:102F6500F010A42417F582E5F03469AD82F5168DCD
:102F750017F583E060DA851382851283747FF00587
:102F850013E51370020512EF2450FF851382851295
:102F950083F00513E51370020512F582851283EFA0
:102FA500F030D003E0F4F0E4FF74022517F517E4E0
:102FB5003516F5160513E51370020512851782857A
:102FC5001683A3E0851382851283F00513E513703C
:102FD500020512851782851683A3E0645585138241
:102FE500851283F020D012851782851683A3E0F41D
:102FF5006455851382851283F00FBF08AC7F1322B9
:06300500E49067E2F0FF19
:01300B0022A2
:10285A00201D03022978E4906478F03010179067FD
:10286A00E3E054F0FFBF50047F2180027F059064AB
:10287A0079EFF080159067E3E054F0FFBF50047FD2
:10288A000980027F02906479EFF090667CE09064A0
:10289A007AF0301006A37414F0800690647B7401F9
:1028AA00F020100302294AE490647CF0906479E0F5
:1028BA00D3940540689067E3E0540FFF1475F0085D
:1028CA00A4FF7D057E02EED394104003022973AC67
:1028DA00050D74782CF582E43464F5837450F0ACF9
:1028EA00050D74782CF582E43464F583EFF0AC05B9
:1028FA000D74782CF582E43464F583E4F074E32EE5
:10290A00F582E43467F583E0FCAB050D74782BF5AA
:10291A0082E43464F583ECF00E0E0F80A990647D96
:10292A007410F09067E3E0541F1490647EF0E4A3FF
:10293A00F09067E5E0FF123CA1906480EFF08029F7
:10294A00E4FD906479E0FFEDC39F501DED25E0247E
:10295A00E3F582E43467F583E0FF747C2DF582E4C5
:10296A003464F583EFF00D80D9C21D7F01227F0008
:01297A00223A
:1018FF0030172DC3E5489564FFE5479563FED3EF99
:10190F009440EE940040197B087D40AF64AE6312A3
:10191F002D7BE5642440FFE43563540FF5638F643A
:10192F0020195C30133FE5605438655B6027E55B39
:10193F0024085438F55B131313541F244BF8E6FF98
:10194F000511E511AC107002051014F5828C83EFB0
:10195F00F0151A80D1E51A6003021A7AD227D2192C
:10196F00C213021A7A302703021A7AD213751A0495
:10197F00301203751A127510677511E3021A7AC2C5
:10198F00199067E3E0F030D00EA3E0F4FF9067E327
:10199F00E06F6012021A509067E4E0FF9067E3E097
:1019AF006F6003021A509067E3E054F0FFBF5004DA
:1019BF007F0880027F01E4FEEEC39F5057EE25E0C3
:1019CF0024E5F582E43467F583E0F020D023EE259B
:1019DF00E024E6F582E43467F583E0F46455FDEE28
:1019EF0025E024E5F582E43467F583E06D705280DD
:1019FF0020EE25E024E6F582E43467F583E06455B4
:101A0F00FDEE25E024E5F582E43467F583E0B505C6
:101A1F00300E80A4D21D906691E0FCA3E0FDA3E000
:101A2F00FEA3E0FFE4FAF9F8EF2401FFEA3EFEE936
:101A3F003DFDE83CFC9066911217C1A212B39212C1
:101A4F0022906699E0FCA3E0FDA3E0FEA3E0FFE493
:101A5F00FAF9F8EF2401FFEA3EFEE93DFDE83CFC10
:101A6F009066991217C1A212B39212301B78E561DA
:101A7F00655C6048E56124085438FFE55C54386FB5
:101A8F0060047E0180027E00E51B60047D01800200
:101A9F007D00EE5D7003021B550513E513AC12704C
:101AAF0002051214F5828C83E0FEE56113131354C3
:101ABF001F2453F8A6068F61151B80B8C21BC211D5
:101ACF00906695E0FCA3E0FDA3E0FEA3E0FFE4FA3F
:101ADF00F9F8EF2401FFEA3EFEE93DFDE83CFC90FA
:101AEF0066951217C122E4F51B7512687513631200
:101AFF0030C18F1B122F55EF251BF51BE51B6418EB
:101B0F007044200B127E1D7F3D122A7F7E687F63FB
:101B1F00E4FB7D18122D7B7512687513630513E5B1
:101B2F0013AE127002051214F5828E83E0FFE56189
:101B3F00131313541F2453F8A607E56124085438D0
:061B4F00F561151BD21B1D
:011B5500226D
:0B3CEB00301C05C21C7F01227F00225C
:10300C00E4FF0F2407F582E43461F5837408F00FB4
:10301C0074072401F582E43461F583E4F07C667D69
:10302C0094FEED1DAA0470011CF5828A83E0FBAAB4
:10303C00070F74072AF582E43461F583EBF00EBEBA
:10304C0004E07C667D98E4FEED1DAA0470011CF57D
:10305C00828A83E0FBAA070F74072AF582E43461A5
:10306C00F583EBF00EBE04E07C667D9CE4FEED1D6A
:10307C00AA0470011CF5828A83E0FBAA070F74076F
:10308C002AF582E43461F583EBF00EBE04E07C6635
:10309C007DA0E4FEED1DAA0470011CF5828A83E07C
:1030AC00FBAA070F74072AF582E43461F583EBF071
:0430BC000EBE04E060
:0130C00022ED
:033D0000C2AE222E
:1033F7000208B0E493A3F8E493A34003F68001F234
:1034070008DFF48029E493A3F85407240CC8C333D6
:10341700C4540F4420C8834004F456800146F6DFA5
:10342700E4800B0102040810204080903C3EE47EBB
:10343700019360BCA3FF543F30E509541FFEE4939A
:10344700A360010ECF54C025E060A840B8E493A361
:10345700FAE493A3F8E493A3C8C582C8CAC583CA8C
:10346700F0A3C8C582C8CAC583CADFE9DEE780BE44
:013C5900006A
:10168E00BB010689828A83E0225002E722BBFE025A
:09169E00E32289828A83E493228D
:1016A700BB010CE58229F582E5833AF583E02250F8
:1016B70006E92582F8E622BBFE06E92582F8E22242
:0D16C700E58229F582E5833AF583E493225C
:1016D40075F008758200EF2FFFEE33FECD33CDCCCD
:1016E40033CCC58233C5829BED9AEC99E582984050
:1016F4000CF582EE9BFEED9AFDEC99FC0FD5F0D62D
:10170400E4CEFBE4CDFAE4CCF9A88222B800C1B956
:101714000059BA002DEC8BF084CFCECDFCE5F0CB94
:10172400F97818EF2FFFEE33FEED33FDEC33FCEBCD
:1017340033FB10D703994004EB99FB0FD8E5E4F988
:10174400FA227818EF2FFFEE33FEED33FDEC33FC75
:10175400C933C910D7059BE99A4007EC9BFCE99A69
:10176400F90FD8E0E4C9FAE4CCFB2275F010EF2FAE
:10177400FFEE33FEED33FDCC33CCC833C810D707AE
:101784009BEC9AE899400AED9BFDEC9AFCE899F8E9
:0E1794000FD5F0DAE4CDFBE4CCFAE4C8F9227C
:0E17A200C3E49FFFE49EFEE49DFDE49CFC2258
:1017B000EB9FF5F0EA9E42F0E99D42F0E89C45F08F
:0117C0002206
:0C17C100ECF0A3EDF0A3EEF0A3EFF0229B
:1017CD00A8828583F0D083D0821217E41217E41219
:1017DD0017E41217E4E473E493A3C583C5F0C5833E
:1017ED00C8C582C8F0A3C583C5F0C583C8C582C866
:0117FD0022C9
:10133200E53A242EF8E6053A22782B302502782E5B
:10134200E475F00112185F02168E201EEB7F2ED27A
:101352001E8018EF540F2490D43440D4FF30220B57
:10136200EF24BFB41A0050032461FFE53B6002156D
:101372003B053EE53E7002053D30250D782BE475B8
:10138200F00112185FEF0217FE0239FD7403D22535
:101392008003E4C225F53A8B2B8A2C892DE4F53B98
:1013A200F53DF53EE53B60077F2012136D80F57534
:1013B2003CFFC21FC21EC220C221C223C224C226B7
:1013C20012133BFF700D3025057F0012137EAF3ED6
:1013D200AE3D22B4255FC2D5C22212133BFF24D0F8
:1013E200B40A00501A75F00A783B30D50508B6FFEA
:1013F2000106C6A426F620D5047002D22180D92483
:10140200CFB41A00EF5004C2E5D22202157ED21FD9
:1014120080C6D21E80C0D22080BCD2D580BAD22350
:1014220080B47F2012136D2020077401B53B004069
:10143200F1121332FF12136D0213A6D226D22480A8
:1014420095121332FB121332FA121332F94A4B700D
:1014520006794F7A167BFF20202EE53B602A7E001C
:101462008E827583001216A760060EEE653C70F040
:10147200C2D5EBC0E0EAC0E0E9C0E0EE1215C5D08B
:10148200E0F9D0E0FAD0E0FB12168EFF60AAEBC0C2
:10149200E0EAC0E0E9C0E012136DD0E02401F9D027
:1014A200E03400FAD0E0FBE53C0460DCD53CD980B6
:1014B200877BFF7A1579C1D220809C7910800279CE
:1014C20008C224C2268008D2D5790A8004790AC2C9
:1014D200D5E53C047002F53CE4FAFDFEFF1213323E
:1014E200FC7B08201F13121332FD7B10301E0A12E0
:1014F2001332FE121332FF7B20EC3382D592D55089
:1015020013C3E4301E069FFFE49EFEE4201F039DEA
:10151200FDE49CFCE4CBF8C21FEC700CCFCECDCC2A
:10152200E824F8F870F38017C3EF33FFEE33FEEDD3
:1015320033FDEC33FCEB33FB994002FB0FD8E9EBB4
:10154200301F05F8D0E0C448B21FC0E00AEC4D4E8F
:101552004F78207B0070C2EAB53C0040BCC0E0126C
:1015620015C7D0F0D0E0201F04C4C0E0C4B21FC031
:10157200F0121356D0F0D5F0EB0213A61218BE14D7
:10158200435314BD5814144C14104214C14F14C9BF
:0F1592004414C94914294314CF5514B34614B354
:1015A1004514B347166F5014182D141C2E143F2BDD
:1015B100142023143D2016582A13D848000014374C
:1015C1003F3F3F00790AA2D5202114302309B910E9
:1015D100020404B9080104A2D52024025001042008
:1015E10020689220B53B005034C0E07F20302119A3
:1015F1007F30A22072247223500F12161EC220C205
:1016010024C223C2267F30800F302303E9C0E012B9
:10161100136D302303D0E0F9D0E0B53BCC30231774
:101621007F30B9100C12136D7F583022077F7880FC
:1016310003B9080312136D3020057F2D02136D7F4E
:10164100202026F87F2B2024F322922080CF286EA1
:10165100756C6C2900D21F121332301FF8C21F782B
:101661003B30D50108F60213D82D504349581213C7
:10167100322403B405004001E490166A9312135E0C
:0D168100743A12135ED221753B040214BDB1
:102114008B2E8A2F8930E4F53AF539F538F537F501
:1021240035F536E532453345316012EBC0E0EAC09F
:10213400E0E9C0E0AB31AA32A93312186FAB2E0527
:1021440030E530AA2F7002052F14F912168EF53BD4
:10215400C394094007E53BD3940D40E1E53B64207B
:1021640060DBE53BB42D054336038016E53BB42B19
:1021740005433601800C74FF2530F53074FF352F8C
:10218400F52FE53460046410703FAB2EAA2FA930FC
:1021940012168E64306009E534702E75340A802975
:1021A4009000011216A7FF64786004EFB45813433B
:1021B400360175341074022530F530E4352FF52FCF
:1021C4008007E5347003753408AB2E0530E530AA7A
:1021D4002F7002052F14F912168EF53BC39461403B
:1021E4000AE53BD3947A5003533BDF74D0253BF587
:1021F4003BC3940A400CE53B9411406D74F9253BB4
:10220400F53BE53BD395345060433601853A3F8531
:10221400393E85383D85373CAF347E00E4FCFDAB68
:102224003AAA39A938A837121810C8ECC8C9EDC998
:10223400CAEECACBEFCBE4FCFDFEEB253BF53AEE50
:102244003AF539ED39F538EC38F537AF3AAE39AD02
:1022540038FCAB3FAA3EA93DA83CD31217B05003AB
:102264000221CD4336040221CDE53620E003E4808B
:102274002DE53245334531601EAB2EE53024FFF9A0
:10228400E52F34FFFAEBC0E0EAC0E0E9C0E0AB318F
:10229400AA32A93312186FE53630E20774FFFFFE45
:1022A400FDFC22E536AF3AAE39AD38AC3730E10348
:0422B4000217A22249
:1017FE00BB010689828A83F0225002F722BBFE01CA
:02180E00F322C3
:10181000E88FF0A4CC8BF0A42CFCE98EF0A42CFC77
:101820008AF0EDA42CFCEA8EF0A4CDA8F08BF0A4F5
:101830002DCC3825F0FDE98FF0A42CCD35F0FCEB54
:101840008EF0A4FEA9F0EB8FF0A4CFC5F02ECD3919
:0F185000FEE43CFCEAA42DCE35F0FDE43CFC2286
:10185F00FAE6FB0808E6F925F0F618E6CA3AF6228A
:10186F00BB011A89828A83D0F0D0E0F8D0E0F9D09A
:10187F00E0FAD0E0FBE8C0E0C0F00218ED5016E946
:10188F00F8D083D082D0E0F9D0E0FAD0E0FBC0826C
:10189F00C0830218E4BBFE16E9F8D083D082D0E0F3
:0F18AF00F9D0E0FAD0E0FBC082C0830218F62225
:1018BE00D083D082F8E4937012740193700DA3A3B9
:1018CE0093F8740193F5828883E4737402936860CD
:0618DE00EFA3A3A380DFCD
:0918E400EBF608EAF608E9F62229
:0918ED00EBF0A3EAF0A3E9F022FC
:0918F600EBF208EAF208E9F22223
:00000001FF
